:03000000021BB12F
:0C1BB10078FFE4F6D8FD7581DD020036F7
:0100190022C4
:0618B7008B318A328933F7
:1018BD007577027F48121A2E121BFDEF20E0F9AB4F
:1018CD0031AA32A933120548787FE6FE08E6FDED10
:0118DD00FF0B
:0118DE0022E7
:100F7B0043525354005341564500434647002D3EC0
:100F8B0053320052415445434C5220554E49544222
:100F9B004C4E4B545249475452455653545254534A
:100FAB00544F505A45524F44464C54534156455258
:100FBB00535420535720202E3173202E3273202E62
:100FCB00357320317320203273202035732020316C
:100FDB0030732033307320316D2020326D2020355B
:100FEB006D202031306D2033306D20316820200092
:100FFB0000000100020005000A0014003200640129
:10100B002C025804B00BB8177046508CA04665657F
:10101B0074596172644D6574724F6666204F6E2011
:10102B00204E6F2020596573204F66662054696DE2
:10103B0065416C7420547269674F66662054696D04
:10104B0065416C74204F66662054726967507772E5
:05105B00205265632036
:10192D0025E024FAF582E4340FF583220533E533FF
:10193D00C394022208F608F608F62275F004A424D2
:05194D0024F9741022D2
:10145200789F76AB0876CD08760008760AE408F61F
:1014620008760108F608766408764012194108F6F3
:1014720078ADF608760A08F608763C08F60876147F
:1014820008F608760F1219417BFF7A0F797B121842
:09149200017F05121763021861C5
:1018DF00757B1D757CC012156A78A0E664CD700407
:1018EF0018E664AB600312145278B9E6FFF4600394
:0718FF00EF700478B97601D7
:0119060022BE
:0D1B7900C2AF7DC07C1DE4FF121AD2D2AFB6
:011B8600223C
:10156A00753EFF857B3F857C40754100754200755D
:10157A00439FE4FFAB3EAA3FA9408F8275830012C6
:10158A00051BAB41AA42A9438F8275830012055AF3
:10159A000FBF1CE078B8E6FFF46003EF700478B878
:0215AA007601C8
:0115AC00221C
:101861007D01E4FF1219D67BFF7A0F7980121801EE
:10187100121B79C2AF7F9F7B1C7DC07C1D121ADCBD
:0D188100D2AF7F02121763E4FDFF0219D6FB
:10097B00E4F5317BFF7A0F79851218017F05121789
:10098B0063A297829650FAA2969217A2979218E5B5
:10099B003175F004A4248EF9740F35F0FA7BFF1235
:1009AB0018017F05121763853132E4F5337BFF7A2B
:1009BB000F7989121801E531B4090050779009CFEE
:1009CB00F82828730209EA020A3F020A0B020A13EB
:1009DB00020A17020A1F020A27020A2F020A377F8E
:1009EB0001EF12192D78A1E6FC08E6FD7401936D59
:1009FB007003E4936C70028F330FBF0FE4020AC2D3
:100A0B0078A3E6F533020AE878A4800278ACE6F521
:100A1B0033020B0278ABE6F533020B2978B5E6F51A
:100A2B0033020B4678B6E6F533020B6378B7E6F57F
:100A3B0033020B80E5316532600302099AA217304D
:100A4B009601B35013A296921730960C0531E531EF
:100A5B00C3940C4003E4F531A218309701B350D482
:100A6B00A29792183097CDE531B40C0050C6900A7E
:100A7B0080F8282873020AA4020AD0020AD6020AB6
:100A8B00F4020B08020B1B020B34020B51020B6E10
:100A9B00020B94020B9A020BA00533E533C3940FA0
:100AAB004003753301E53312192DE493FF74019361
:100ABB0078A1CFF608EFF6E53375F004A424BEF960
:100ACB00740F020B8912135C020A3F0533E533C323
:100ADB0094034003E4F53378A3A633E53375F004B0
:100AEB00A42418F97410020B891219394003E4F588
:100AFB003378A4A633E533121948020B891219393E
:100B0B004003E4F53378ACA633E533121948806E15
:100B1B001219394003E4F53378ABA633E53375F09E
:100B2B0004A4242CF9741080550533E533C39404C5
:100B3B004003E4F53378B5A633E53375F004A4240C
:100B4B0034F9741080380533E533C394034003E460
:100B5B00F53378B6A633E53375F004A42444F97461
:100B6B0010801B0533E533C394044003E4F533785D
:100B7B00B7A633E53375F004A42450F9741035F09F
:100B8B00FA7BFF121801020A3F121452020A3F129B
:0B0B9B001861020A3F43A208020A3F53
:0A1BC9004552415300444F4E4500C1
:101B480078A1E6F55508E6F55622E56CAE6B780601
:011B5800226A
:10112600C215C21678B9E6C43354E0FEE4F5728EF1
:1011360071F570F56F7B40FAF9F8AF72AD70AC6F70
:101146001206078E698F6AE4F532F533C3E53395E7
:101156006AE5329569501CE53164816016AF33AE9D
:1011660032121833121ABE8F310533E53370DD059E
:101176003280D9E531B48108E53315337002153272
:10118600E533656A7004E5326569700CD215121B89
:1011960095E4F56BF56C800785326B85336CE4F569
:0911A6006DF56E755480121B48B2
:0111AF00221D
:10183300C3EF956AEE95695024EF7806C333CE3330
:10184300CED8F9FD757702EE787FF6CFEDCFEF08AE
:0D185300F67F50121A7C121BFDEF20E0F909
:011860002265
:031A4900CDEFCD11
:101A4C00757702EE787FF6ED08F67F50121A7C124D
:061A5C001BFDEF20E0F984
:011A62002261
:101ABE007577017F50121A2E121BFDEF20E0F97878
:031ACE007FE6FFB1
:011AD10022F2
:101AA900121A49E4FFFE0FBF00010EBE0FF8BFA0D6
:041AB900F5121ABE4A
:011ABD002206
:06179900CBEFCBCAEECA43
:10179F00301503301627757703EA787FF6EB08F6D6
:1017AF0008EDF67F50121A7C121BFDEF20E0F9E4D2
:0D17BF00FFFE0FBF00010EBE0FF8BFA0F52A
:0117CC0022FA
:1015F000753400753500753654E4F533121B52C34B
:1016000033CE33CED8F97C002533FFEC3EFEAB342D
:10161000AA35A93685338275830012051BFD121782
:10162000990533E533C3940640D2756D00756E0697
:011630002297
:1011B0008E318F32121B52C333CE33CED8F9256E07
:1011C000FFE56D3EFEEEC0E0EFC0E0E531FDD0E0B2
:1011D000FFD0E0FE121799056EE56E7002056D12E4
:1011E0001B52C333CE33CED8F9256EFFE56D3EFEDC
:1011F000AD32121799056EE56E7002056D0558E562
:101200005870020557C3E56E9440E56D9400401791
:10121000E4F56DF56E056CE56C7002056B956AE59D
:081220006B95694002D2152212
:10135C00E4F56DF56E7BFF7A1B79C9121801D21674
:10136C00E4F53EF53FC3E53F956AE53E95695021AE
:10137C00E53FAE3E7806C333CE33CED8F9F56E8E4C
:10138C006D7D81FF121799053FE53F70D8053E80B2
:10139C00D4C2167BFF7A1B79CE121801E4F56BF5DB
:0713AC006CF56DF56EC21532
:0113B3002217
:10130300E4F53EF53FF540F541C3E541956AE54017
:1013130095695044E53F6481603EAF41AE40121889
:1013230033121ABE8F3FE53F64807022AF3E053E05
:10133300FCFDFEFBFAF9120D527F2C120016AE4093
:10134300AF41E4FCFDFBFAF9120D52121BE6054115
:08135300E54170B5054080B1D1
:01135B00226F
:02149B008F3E82
:10149D00E4F53FF540F541F542C3E542956AE54176
:1014AD0095695030E5406481602AAF42AE41121813
:1014BD0033121ABE8F40E540B4800FE53F653E7094
:1014CD0007AF42AE41021833053F0542E54270C9F0
:0414DD00054180C580
:0114E10022E8
:10163100121B4878ACE6F559E4F557F5581215F048
:10164100856B73856C747F0112129F30021A78AF1B
:10165100E6FE08E6FFE4FCFD7B64FAF9F812057C7E
:101661008F668E658D648C63300505C205121A93F1
:011671002256
:10172900856B31856C32E56E456D60080532E532B1
:101739007002053185736B85746C1215F085316BF8
:1017490085326CC3E532956AE53195694007E4F560
:0A1759006BF56CD2157F0202129F9F
:101AD200740478FF769612FF0322740078FF7696DC
:041AE20012FF0322CA
:0300330002106058
:0D106000C0E0C0F0C083C082C0D075D008D1
:10106D00E5D954F8FF120720109A08109A1010A90C
:10107D001810C42010AB2810C43010C63810CC4046
:10108D0010C44810E55011025800001110857ADA8D
:10109D00C2DDC2DC7578007579008070800EE57751
:1010AD00700280560579E579700205781200268F59
:1010BD00DAC2DDC2DC80558016D2DDC2DC804DC2C5
:1010CD00DDC2DCE5777004C2DA8041D2DA803DC240
:1010DD00DDD2DC7575048034AFDA121BBD0579E500
:1010ED007970020578C2DDC2DCE5777004C2DA8062
:1010FD001BD2DA8017AFDA121BBDC2DDD2DC7575DB
:0E110D00028009757504C2DDC2DCD2DAC2DBD5
:0B111B00D0D0D082D083D0F0D0E032E2
:10188E0043910C43920CE4F5DBEF25E0F5DB3017CA
:10189E000343DB0175DD2575DC2575D84453F8FE51
:0918AE0053F7FEE4F575D2E822BF
:101A7C00E57530E002FF22E4F576757503EF25E09D
:071A8C00F57AD2DD7F022292
:101A2E00E57530E002FF22E4F5761577757505EF62
:0B1A3E0025E04401F57AD2DD7F022292
:061BFD0020DBFDAF7522A4
:0D0026001577AF760576747F2FF8E6FF2280
:0C1BBD00747F2576F8EFF6057615772288
:0E1B8700E4F5847585FFF592F5A475A5FF229F
:071BEF00EE3395E0FDFC223E
:10195200C212C214C211D2A2C2A0C2A1E4FDFF12DD
:1019620019D6E4FD7F011219D67F0812129F7F0457
:0319720002129FBF
:1019D600EF146011047016BD0104C2A78002D2A7DD
:0E19E600A2A7921322BD0103C2A622D2A622FE
:10129F00EF14B40800505C9012B475F003A4C5832A
:1012AF0025F0C583730212CC0212D20212D9021298
:1012BF00E50212E70212E50212F10212F9D21275DB
:1012CF00190122C212A21392A722D214751A057DF8
:1012DF00017F010219D68005C211C28722C211D225
:1012EF008722D211D28775180122C2A47F0112174B
:0412FF0063D2A422F0
:1016B100301212D5190F30A707C2A775191E800560
:1016C100D2A7751946E51AD39400400CD51A09C260
:1016D10014E4FD7F011219D6301111D5180E30878F
:0D16E10006C28775180522D28775181E22D3
:10199600C374039FFE1392A0EEA2E192A1AF80CF83
:0F19A6005480CFED547FCF4FCF8F80C2A2D2A2FB
:0119B500220F
:061801008B408A41894280
:10180700E4FCCFECCF7D201219960CBC04F4E4FC69
:10181700AB40AA41A9428C8275830012051BFD606B
:0B1827000ACFECCF1219960CBC04E5B0
:011832002293
:041228008F828E83A0
:10122C00121BEFE47B0F7A27F9F8C31206A75003C1
:10123C0090270FAF82AE83121BEF7B197AFC79FFDC
:10124C0078FFD31206A7400390FC19E4F531741B08
:10125C002531F8E4F60531E531B405F2AE83AF8201
:10126C00121BEF7B007A00791B120D52E51E701ACF
:10127C00753103741A2531F8E6FF741B2531F8C655
:10128C00EFC6D531EE751B2080E27B007A00791B0E
:03129C0002180134
:1019F40046554C4C0050524F47005A4C4F47004DEF
:0D1A04004F440076322E370054726967009F
:101B2200E6FE08E6FFE4FCFD2278D61206E278CE55
:031B32000206FBAD
:030013000219755A
:10197500C0E0C0D075D010200E0CAF8DEFAD8BF54B
:101985005EEDF55FD20E758D00758B00D0D0D0E081
:01199500321F
:021763008F3FB6
:10176500E4F540F541C3E541953FE540940050233C
:10177500900000AF82AE83E4FCFD7B207A4EF9F841
:10178500D31206A74003A380EA0541E54170D605BB
:031795004080D2BF
:01179800222E
:0E1B95007BFF7A1979F41218017F0A02176398
:0F1B6A00D20B301506121B95C20B221216312218
:05000E00C20B021729DE
:101A930078DA12070700000000121B2B78D6120712
:061AA30007000000002214
:10003600121B87121BD31219527F041217632097C3
:10004600127BFF7A1979F91218017F011214E2D294
:10005600AF80FE209612D2AF1218DFC2177F701241
:10006600188E12112612097B7A1979FE1204F7E40A
:10007600FF1214E2D2AF1218DF7BFF7A1A7903124D
:10008600180178B8E62430FD7F031219967F041212
:1000960017637A1A79071204F7C2177F7012188E3F
:1000A6007F01121763121126120019C21A1216EED8
:1000B6007F01121763E4F560F56112001AA29692A9
:1000C60008A2979209E4F52478D2120707000000E7
:1000D60000E4F52578DA120707FFFFD8F178CE128B
:1000E600070700000000E4F55378D6120707000062
:1000F6000000C20DC20BC20CE4F567F568F526F5E3
:1001060027F55EF55FC20EF562C20FF55DF55CF58B
:100116005BF55AF566F565F564F563F52078B5E6A1
:1001260024FE600B14600C2402700AD2018006D2F1
:10013600068002D20078B6E624FE6007047006D276
:10014600028002D20778B7E624FE600B14600C2406
:1001560002700AD2038006D2048002D2053001174B
:10016600C20178AD121B227B64FAF9F812057C8F66
:100176005D8E5C8D5B8C5A301AFDC21A300C33A230
:1001860008309601B3400BA209309701B340030231
:10019600026430961230970FC20CE4F567F5687F5B
:1001A6000412129FE4F553A2969208A297920902AE
:1001B6000264209605209702D21030965630975347
:1001C600301031C21078CE1206E2EC4D4E4F78DA7E
:1001D600700C12070700000000121B2B801012077C
:1001E600070000000078CE12070700000000D209C1
:1001F600D208802478A4E6601F0568E568700205C9
:1002060067D394B8E567940B400ED20C7F051212A3
:100216009F8005E4F567F568A208309601B3501F84
:10022600A2969208309618201015C201E553600771
:10023600E4F5537F0680057553017F0712129FA2CE
:1002460009309701B35017A29792093097102010E2
:100256000DB20B300B05121B6A800312000E12073B
:1002660046AF5DAE5CAD5BAC5AEC4D4E4F6026744E
:10027600FF2FF55DEE34FFF55CED34FFF55BEC34F6
:10028600FFF55AAF5DAE5CAD5BFC4D4E4F70062080
:100296000B03121B6AAF66AE65AD64AC63EC4D4EE4
:1002A6004F602374FF2FF566EE34FFF565ED34FFDE
:1002B600F564EC34FFF563AF66AE65AD64FC4D4E98
:1002C6004F700312000E200E03020374C2AFC20E5B
:1002D600D2AFE4855F30855E2FF52EF52DAF30AEBB
:1002E6002FAD2EAC2D7B107A27F9F812057C8F30B6
:1002F6008E2F8D2E8C2DE4FB7A90F9F81215268F11
:10030600308E2F8D2E8C2D78ABE66009C374B89F86
:10031600FF740B9EFEE56214601624FE6020240323
:100326007049C3EF94B0EE9404500E7562018009D3
:10033600D3EF9414EE940540357562038030C3EF15
:1003460094B0EE94045027756201300006200B032A
:10035600121B6A300305C203121A93300B02D20F26
:100366007BFF7A1A790C1218018003E4F5620525E1
:10037600E525C3940250030204F1E4F525FB7A0057
:1003860079281218B78E298F2AE52864026003029D
:1003960004F178D21206EEE8C0E0E9C0E0EAC0E077
:1003A600EBC0E078A3E6FDAF2AAE29121406D0E032
:1003B600FBD0E0FAD0E0F9D0E0F8EB2FFFEA3EFE02
:1003C600E93DFDE83CFC78D21206FB0524E524C392
:1003D600940550030204F178D21206E2E47B05FA92
:1003E600F9F812152678D21206FB78D21206E278B0
:1003F600CE1206EEC3EF9BFFEE9AFEED99FDEC984A
:10040600FC78D21206FB78DA1206E278D21206EEF1
:10041600D31206A7400A78D21206E278DA1206FB51
:10042600E553600A78DCE6FE08E68E2BF52C78D4D8
:10043600E6FE08E68E29F52AE5536006AF2CAE2BBC
:100446008004AF2AAE291212280527E52770020577
:1004560026C378A296E52618964040E4F526F527A9
:10046600300D0DE529FF120016AF2AE52A120016F7
:10047600300B287F0312129F20151A78ACE6600C09
:10048600300F097F007E821211B0C20FAF2AAE294B
:100496001211B08006121B9512000E78D21206E2D7
:1004A60078D61206FB78D212070700000000E4F5A2
:1004B60024300405C204121A9330061678B1121BB2
:1004C6002278D61206EED31206A74006200B031298
:1004D6001B6A30071678B3121B2278D61206EEC3B3
:1004E6001206A75006300B0312000E1216B10201B7
:0104F6007D88
:0B04F7007BFF1218017F041217632224
:10190700444C0021536967005A4C4F47004D4F44E0
:1019170000322E37004A616E2030372032303035A2
:061927000050524F470082
:1015AD00AF39AE38AD37AC36EC4D4E4F22EF24FF90
:1015BD00F539EE34FFF538ED34FFF537EC34FFF542
:1015CD003622E475392075384EF537F53622E47537
:1015DD003901F538F537F536227533007534007558
:0315ED00359F2205
:10074600121BA3EF700302095B7F0412129FE4F5EC
:1007560053C20CF567F568121A11EF120720093F0C
:100766002409482A094B50089852078C61081A63D5
:10077600086D6C087372087073089C74090F76090B
:1007860007780000095B7BFF7A19790712180112B6
:1007960015CF121BA3EF700A1215AD60051215BA1C
:1007A60080F01215AD700302095B121A118F321216
:1007B600149BE4F5391215DFE47F06FEFDFCAB3928
:1007C600AA38A937A836C31206BD501F121ABE8F03
:1007D60032120016E5392401F539E43538F538E4E6
:1007E6003537F537E43536F53680CD121ABE8F32F9
:1007F600E53264806016E5326481601012001612DC
:100806001ABE8F321200167531018003E4F531E508
:100816003170D8221215E61215DBF5321215AD60CD
:10082600241215CF121BA3EF700A1215AD60051224
:1008360015BA80F01215AD600312095C0532E53277
:10084600C3941C40D71215AD601A789FB6AB070843
:10085600B6CD030209457BFF7A19790A1218017F82
:100866000A021763020904B20D220213031215E6E7
:10087600E4F532AB330535E535AA34700205341498
:10088600F9120502FF1200160532E532C3941C4028
:10089600E22243A2082275330075340075357D12B5
:1008A60015DBF5321215AD60241215CF121BA3EF1E
:1008B600700A1215AD60051215BA80F01215AD60FA
:1008C6000312095C0532E532C3940240D71215AD16
:1008D600602CAE7DAF7EEE3395E0FDFC78D6120639
:1008E600EEC3EF9BF53DEE9AF53CED99F53BEC98A2
:1008F600F53AAF3D78A9E53CF608EFF680410215DA
:100906006A7F0412129F02135C7A19790F1209701A
:100916007A197914121B3578B8E62430FF120016BE
:10092600121BE67F761200167A1979181209707A68
:1009360019791C121B35021BE6E478A9F608F602A3
:1009460018610214527BFF7A1979281218017F0167
:050956001214E280FE16
:10095B0022121A11AB33AA34A93585328275830062
:10096B00EF12055A227BFF121B35121BE67BFF226F
:0A1BD300E4F5955396BF53A27F225C
:1016EE005389F0438901538FFE758C70E4F58A534C
:1016FE00B8FD53B7FDD2A9D28C53890F43899053AD
:10170E008FEFF58DF58B4391105392EF53B8F7533E
:0B171E00B7F7D2ABD28ED28AD2AA223B
:03000B00021BDDF8
:091BDD00D21A758C70758A003271
:03001B00021BF6CF
:071BF600758D00758B0032B4
:101AE6000D0A003031323334353637383941424306
:041AF600444546001D
:101AFA00AF52AB46AA47A948055222AF45AE44ADFC
:041B0A0043AC422284
:1014E2005387BF75985053877FE4F5BABF01054310
:1014F200A240800353A2BFE4F5BD75BE30F5BF75AF
:10150200BD035391FE4392014391025392FDC21BCC
:1015120053B8EF53B7EF43B81078CCF618F678CD3E
:04152200F6D2AC222F
:030023000217CDF4
:1017CD00C0E0C0D075D01030981E78CCE6C3940F11
:1017DD00501418E60624BBF8A69978CC0618E6C373
:1017ED00941040027600C298309904C299C21BD061
:0417FD00D0D0E03236
:08000300201BFDD21B8F992286
:1019B60078CCE6D39400401508E60624BBF8E6FF8B
:0F19C60078CC1608E6C394104005E4F6227F00A3
:0119D50022EF
:03001600020003E2
:101A11007F207E4E78CCE67010D3EF9400EE9400D8
:0C1A21004007EF1F70EE1E80EB1219B69C
:011A2D002296
:101B3500120502FF600C120016740129F9E43AFA45
:031B450080EE220D
:0E1BA30078CCE6D3940040037F01227F00221D
:101A6300CEEFCEEE54F0C4540F901AE993FF120058
:091A730016EE540F93FF02001659
:101B5900CDEFCDCCEECCEEFF121A63CFEDCF021A4A
:011B69006318
:091BE6007BFF7A1A79E6021B3537
:0E0D52008F458E448D438C428B468A478948DC
:100D6000E4F552EC4D4E4F7017E94A4B70057F3059
:100D7000020016121AFA8F827583007430020E7503
:100D8000121B07EC33502AE5484547454670077F5C
:100D90002D120016800D121AFA8F82758300742DA1
:100DA00012055A121B051206998F458E448D438CED
:100DB00042755101754C00754BCA754A9A75493B8D
:100DC000E4FFFEFDFCAB4CAA4BA94AA849D312068E
:100DD000BD5003020E60121B05A8491206078F5072
:100DE0008E4F8D4E8C4DEC4D4E4F7004E55170235F
:100DF000E5502430FFE5484547454670051200168A
:100E0000800EAE52121AFC8E82758300EF12055AC4
:100E1000E4F551AF4CAE4BAD4AAC49AB50AA4FA92B
:100E20004EA84D12057CC8ECC8C9EDC9CAEECAC3AC
:100E3000E5459FF545E5449AF544E54399F543E5D5
:100E40004298F542AF4CAE4BAD4AAC49E47B0AFA4E
:100E5000F9F81206078F4C8E4B8D4A8C49020DC053
:100E6000E547454845466010AB46AA47A948855224
:080E700082758300E412055AAB
:010E78002257
:100BA6000134C35001DBBF68028BBB800344B79896
:100BB6000407B3B004D5AFC805A9ABE00689A7F80A
:100BC6000775A410086DA02809719C400A819858E1
:100BD6000B9F94700CCA90880DE98CF90E048CA0BA
:100BE6000EA88AAC0F4D88B80FF786C410A184D022
:100BF600115182DC120580E812BB7EF413747D006D
:100C060014307B0C14F2791815B8772416807530D9
:100C1600174B733C1819714818ED6F5419C46D6061
:100C26001AA16B6C1B7E69781C6167841D4A6590EE
:100C36001E37639C1F2561A8201A5FB421125DC070
:100C4600220D5BCC230E59D8241557E4251F55F0E9
:100C5600262F53FC27425208285B501429764E2033
:100C66002A9B4C2C2BC04A382CEE48442E1E46504C
:100C76002F55445C308F426831D1407433173E8023
:100C860034633C8C35B13A98370938A4386636B0A7
:100C960039C734BC3B2D32C83C9D30D43E0F2EE0C4
:100CA6003F882CEC41062AF8428D29044418271067
:100CB60045AB251C4741232848E121344A861F407D
:100CC6004C311D4C4DE21B584F9C1964515D1770F9
:100CD6005323157C54EF138856C4119458A20FA0C1
:100CE6005A830DAC5C6D0BB85E6009C4605807D0C2
:100CF600625A05DC646203E8667301F4688A0000E0
:100D06006AA1FE0C6CB8FC186ECFFA2470E6F830B7
:100D160000000000000000000000000000000000CD
:100D260000000000000000000000000000000000BD
:100D360000000000000000000000000000000000AD
:0C0D4600000000000000000000000000A1
:1016720075F004E538A424A6F582E5F0340BF58371
:10168200E49322FE740193FF75F004E538A422F579
:1016920083C37401939FFFE4939EFEE4228F398EED
:0F16A200388D378C36228F358E348D338C322233
:101B0E00C3EF9DEE9C400AD3EF9BEE9A50037F01EC
:041B1E00227F002200
:040E79008E368F37EB
:100E7D00E4F538121672FC740193FD12168A24AA39
:100E8D00F582E5F0340BF583E493FA740193FBAF2F
:100E9D0037AE36121B0EEF7003020F691216721267
:100EAD00168524AAF582E5F0340B1216918F3C8E2F
:100EBD003BF53AF53912168A24ACF582E5F0340B80
:100ECD00F583E49312168524A8F582E5F0340B1210
:100EDD0016918F408E3FF53EF53DAD3EAC3D120671
:100EED00998F408E3F8D3E8C3DAE36AF37E4FCFD85
:100EFD00EEC0E0EFC0E0121672FE740193FBCAEE75
:100F0D00CAD0E0FFD0E0FEC3EF9BFFEE9AFEED945A
:100F1D0000FDEC9400FCAB40AA3FA93EA83D120594
:100F2D007CAB3CAA3BA93AA839121526C8ECC8C916
:100F3D00EDC9CAEECACBEFCB12168A24A8F582E50D
:100F4D00F0340BF583E493FE740193FFE4FCFDEBA9
:100F5D002FFFEA3EFEED39FDEC38FC220538E53871
:0D0F6D00C3946A5003020E80E4FFFEFDFCF9
:010F7A002254
:01001A0022C3
:1013B40012169FAB39AA38A937A836E8C0E078A737
:1013C400E6FE08E6FFE4FCFDD0E0F812057C121608
:1013D4009F780E1206CE12169F78A9E6FE08E6FF45
:1013E400EE3395E0FDFCE5392FF539E5383EF53867
:1013F400E5373DF537E5363CF536AF39AE38AD3730
:02140400FC22C8
:021406008D3126
:10140800120E791216A81213B41216A8E531146038
:101418001C14702DE47FE87E03FDFCAB35AA34A9CB
:1014280033A83212057CE47BE87A0B800CAF35AE2A
:1014380034AD33AC32E47B03FAF9F81215261216F0
:09144800A8AF35AE34AD33AC326F
:011451002278
:10050200BB010689828A83E0225002E722BBFE02F7
:09051200E32289828A83E493222A
:10051B00BB010CE58229F582E5833AF583E0225095
:10052B0006E92582F8E622BBFE06E92582F8E222DF
:0D053B00E58229F582E5833AF583E49322F9
:10054800BB010689828A83F0225002F722BBFE0192
:02055800F3228C
:10055A00F8BB010DE58229F582E5833AF583E8F0D7
:10056A00225006E92582C8F622BBFE05E92582C883
:02057A00F2226B
:10057C00E88FF0A4CC8BF0A42CFCE98EF0A42CFC1E
:10058C008AF0EDA42CFCEA8EF0A4CDA8F08BF0A49C
:10059C002DCC3825F0FDE98FF0A42CCD35F0FCEBFB
:1005AC008EF0A4FEA9F0EB8FF0A4CFC5F02ECD39C0
:0F05BC00FEE43CFCEAA42DCE35F0FDE43CFC222D
:1005CB0075F008758200EF2FFFEE33FECD33CDCCE7
:1005DB0033CCC58233C5829BED9AEC99E58298406A
:1005EB000CF582EE9BFEED9AFDEC99FC0FD5F0D647
:1005FB00E4CEFBE4CDFAE4CCF9A88222B800C1B971
:10060B000059BA002DEC8BF084CFCECDFCE5F0CBAE
:10061B00F97818EF2FFFEE33FEED33FDEC33FCEBE7
:10062B0033FB10D703994004EB99FB0FD8E5E4F9A2
:10063B00FA227818EF2FFFEE33FEED33FDEC33FC8F
:10064B00C933C910D7059BE99A4007EC9BFCE99A83
:10065B00F90FD8E0E4C9FAE4CCFB2275F010EF2FC8
:10066B00FFEE33FEED33FDCC33CCC833C810D707C8
:10067B009BEC9AE899400AED9BFDEC9AFCE899F803
:0E068B000FD5F0DAE4CDFBE4CCFAE4C8F92296
:10152600C2D5E830E70FB2D5E4C39BFBE49AFAE4F0
:1015360099F9E498F8EC30E717B2D512155C120663
:1015460007E4C39BFBE49AFAE499F9E498F880036C
:1015560012060730D50DE4C39FFFE49EFEE49DFD11
:04156600E49CFC22E3
:0E069900C3E49FFFE49EFEE49DFDE49CFC2272
:1006A700EB9FF5F0EA9E42F0E99D42F0EC6480C8CA
:0606B70064809845F0226A
:1006BD00EB9FF5F0EA9E42F0E99D42F0E89C45F093
:0106CD00220A
:1006CE00E86010ECA2E713FCED13FDEE13FEEF1342
:0406DE00FFD8F0222F
:0C06E200E6FC08E6FD08E6FE08E6FF2244
:0D06EE00E6FB08E6F908E6FA08E6CBF8227C
:0C06FB00ECF608EDF608EEF608EFF6222B
:10070700D083D082E493F608740193F608740293B9
:09071700F608740393F6740473F0
:10072000D083D082F8E4937012740193700DA3A368
:1007300093F8740193F5828883E47374029368607C
:06074000EFA3A3A380DF7C
:00000001FF
